:020000040000FA
:04000000EAEF01F032
:08000800ECEF01F01652D8A440
:100010000BEF00F01200FF0E0000000000000000D7
:1000200000000000000000000000000000000000D0
:1000300000000000000000000000000000000000C0
:1000400000000000000000000000000000000000B0
:1000500000000000000000000000000000000000A0
:100060000000000000000000000000000000FF0F82
:10007000D8A40CEF00F00000000000000000000019
:100080000000000000000000000000000000162E2C
:100090000BEF00F01200FA0E166E06EC00F0FA0EEE
:1000A000166E06EC00F0FA0E166E06EC00F0FA0E74
:1000B000166E06EC00F0152EEED71200256A266AA1
:1000C000226A236A246A24B81200D8902236233682
:1000D0001B361C36253626361D50255C1E502662E2
:1000E000265C05E31D50255E1E50265A2280242AD8
:1000F000EAD7236A246A266A276A256A25B8120085
:10010000D890263627361736183623362436195017
:10011000235C1A502462245C05E31950235E1A50B4
:10012000245A2680252AEAD7130414E1020E136EFE
:10013000FB0E9614966EFB0E8414176E040E1710A9
:10014000846EFE0E9414946EFE0E8214826E145011
:10015000116E0BD1020E136233D0030E136EFE0E1E
:100160009414946EFE0E8214176E010E1710826E98
:10017000FB0E9414946EFB0E8214826E1B6A0F5059
:10018000176E1050186E10AE06D0171E181E172AC4
:10019000D8B4182A1B2AE80E196E030E1A6E79ECD1
:1001A00000F02650126E1BA002D0121E122A000E62
:1001B000EA6E050EE96E1250E926EF50116ED5D0A9
:1001C000030E13624FD0040E136EFB0E9414946E44
:1001D000FB0E8214176E040E1710826EEF0E93142E
:1001E000936EEF0E8114816E226A0F50176E1050BD
:1001F000186E10AE06D0171E181E172AD8B4182A6B
:10020000222A640E196E1A6A79EC00F026501F6ECD
:100210002750206E22A005D01F1E201E1F2AD8B4F2
:10022000202A1F501B6E20501C6E20AE05D01B1EB6
:100230001C1E1B2AD8B41C2A0A0E1D6E1E6A5EECF8
:1002400000F02550216E20AE02D0211E212A21501F
:10025000126E000EEA6E050EE96E1250E926EF509E
:10026000116E83D0040E13624FD0050E136EEF0E85
:100270009314936EEF0E8114176E100E1710816E8B
:10028000EF0E9214926EEF0E8014806E0F501B6E64
:1002900010501C6E10AE05D01B1E1C1E1B2AD8B49D
:1002A0001C2A640E1D6E1E6A5EEC00F025501F6E47
:1002B0002650206E10AE05D01F1E201E1F2AD8B457
:1002C000202A226A1F50176E2050186E20AE06D0CA
:1002D000171E181E172AD8B4182A222A0A0E196EB9
:1002E0001A6A79EC00F02650216E22A002D0211E5D
:1002F000212A2150126E000EEA6E050EE96E125090
:10030000E926EF50116E31D0010E136EEF0E9214EC
:10031000926EEF0E8014176E100E1710806EFB0E8B
:100320009614966EFB0E8414846E0F501B6E105044
:100330001C6E10AE05D01B1E1C1E1B2AD8B41C2A16
:100340000A0E1D6E1E6A5EEC00F02550176E10AE90
:1003500002D0171E172A1750126E000EEA6E050EF5
:10036000E96E1250E926EF50116E956A1150836EB6
:1003700012000F0EC16E080E6F6EB60E0F6E050ED8
:10038000106E030E056E9F0E066E250E076E0D0E87
:10039000086E990E096E490E0A6EC10E0B6E1F0E85
:1003A0000C6E190E0D6E0E68D59AD588F00ED51408
:1003B000156E070E1510D56EF28EF28AFE0E146EB3
:1003C000640E166E06EC00F01468010E156E4BEC10
:1003D00000F0F4D7B9EF01F0EACF01F0E9CF02F075
:1003E000F4CF03F0F3CF04F0F2A403D094EC00F0C8
:1003F000F29404C0F3FF03C0F4FF02C0E9FF01C0A0
:04040000EAFF1100FE
:020000040030CA
:0E000000240E3F1E008181000FC00FA00F4094
:00000001FF
